:020000040000FA
:0600000011EF1EF01200DA
:0600080004EF08F01200F5
:060018000CEF08F01200DD
:0610000011EF1EF01200CA
:0610080041EF1CF0120094
:061018004AEF1CF012007B
:06102A000100403C000043
:081030002D0F00000300000079
:08103800D9CFE6FFE1CFD9FF9B
:10104000E652636A626A0F019F0E5D6FFB0E5C6F72
:10105000658C659C5E6B0F0EE66EE66AE66A4D0E69
:10106000E66E0F0EE66EB7EC1DF0146E050EE15E37
:101070001450DF6ADF50146E156A040E145C000E03
:10108000155810E2DF50040DF3CFE9FFF4CFEAFF6B
:10109000000EE926040EEA22EE6AEE6AEE6AEE6AB5
:1010A000DF2AE8D70F01160E4C6F62A60CD0030E94
:1010B000E66E620EE66E0F0EE66E5DEC0FF0E55228
:1010C000E552E552F2D7DF6A020EDF5C04E20F015F
:1010D000146BDF2AF9D765980F01040E0B6F040E0D
:1010E0000C6F016B006BE552E552E7CFD9FF1200A0
:1010F000D9CFE6FFE1CFD9FFE6520F01005114E14D
:1011000006D0656A0F015C6B0F01006B87D0656AC2
:101110000F015C6B65B602D06586FCD70F01010E2E
:10112000006F0F01140E5F6F0F0100050AE165BA31
:1011300008D0626A0F015C6B5C815C890F01020E52
:10114000006F6250040B05E00F015C51040B01E0DD
:101150009ED865B263D06250010B12E00F015C5162
:10116000010B0EE069DF0F01040E006F0401100E89
:10117000026F040E036F080E016F006B8C0E0013DC
:101180006250100B05E00F015C51100B01E06FD8AD
:101190006250400B11E00F015C51400B0DE087ECF9
:1011A0001CF0060EE66E620EE66E0F0EE66E5DEC4D
:1011B0000FF0E552E552E5526250200B05E00F01B9
:1011C0005C51200B01E02FD86250020B07E00F01A9
:1011D0005C51020B03E088EC1CF0636A040E0F0103
:1011E000005D01E21BD00F015CA718D0DF6A040E7E
:1011F000DF5C14E262A60FD064CF1AFF030EE66E26
:10120000620EE66E0F0EE66E5DEC0FF0E552E552F3
:10121000E55251D801D002D0DF2AE9D7E552E55294
:10122000E7CFD9FF12000F014CA115D003CFE9FF82
:1012300004CFEAFFEF5080080DE10BCFE9FF0CCFA0
:10124000EAFFEF50840806E103CFE9FF04CFEAFF8D
:101250008C0EEF6E4C91060EE66E620EE66E0F0E71
:10126000E66E5DEC0FF0E552E552E55212000F011B
:101270005C85040EE66E620EE66E0F0EE66E5DECA9
:101280000FF0E552E552E552658285EF1CF065925C
:1012900086EC1CF00F015C9562A40CD0020EE66E89
:1012A000620EE66E0F0EE66E5DEC0FF0E552E55253
:1012B000E552F2D71200FD0E0F011A151FE17E0E46
:1012C0001A15E8407F0B040DF3CF03FFF4CF04FFA2
:1012D000000E0327040E042303CF05FF04CF06FFEF
:1012E00003CFE9FF04CFEAFFEF503C0BE842E842AE
:1012F0000D0802E109D801D01ED805D0FD0E1A153F
:10130000040801E135D812000BCFE9FF0CCFEAFF4A
:10131000EF50800B05E00BCFE9FF0CCFEAFFEF6A3F
:101320000F010F6B106B156B166B146BFFD889ECEC
:101330001CF06FEF0CF0020E0F01105D17E1A3EC33
:101340000DF003CFE9FF04CFEAFFEF50400B07E1B8
:1013500005CFE9FF06CFEAFFC80EEF6E06D005CF36
:10136000E9FF06CFEAFF880EEF6E01D050D81200D9
:10137000D9CFE6FFE1CFD9FFE6520BCFE9FF0CCF83
:10138000EAFFEF50400B01E0010EDF6E080E0F0187
:10139000005D0DE112C45EFF0F015E51000804E222
:1013A0000F01100E006F03D00F01040E006F100527
:1013B00028E10BCFE9FF0CCFEAFF020EE926000E71
:1013C000EA22180EEE6E040EED6E2FDB020E0F01F8
:1013D0000F5D07E10BCFE9FF0CCFEAFF840EEF6E44
:1013E0000FD0DF5007E10BCFE9FF0CCFEAFFC80EAB
:1013F000EF6E06D00BCFE9FF0CCFEAFF880EEF6E41
:1014000001D005D8E552E552E7CFD9FF1200D9CF78
:10141000E6FFE1CFD9FF030EE126020E0F01105DBA
:101420004AE16550100B47E003CFE9FF04CFEAFF24
:10143000EE52EF50146E156A080E141801E11550A3
:101440003AE103CFE9FF04CFEAFFEF503C0BE8425B
:10145000E8420D0830E105CFE9FF06CFEAFFEF5083
:10146000800B29E105CFE9FF06CFEAFF020EE9264E
:10147000000EEA22100EEE6E040EED6EDF6ADF50F3
:10148000146E156A080E145C000E155813E2DF5036
:10149000EA6A180FE96E040EEA22EF50E66EDF509A
:1014A000EA6A100FE96E040EEA22E552E750EF6E89
:1014B000DF2AE5D731D0106B05CFE9FF06CFEAFF71
:1014C000EE52080EEF6E05CFE9FF06CFEAFF020EDF
:1014D000E926000EEA22100EEE6E040EED6E05CF28
:1014E000E9FF06CFEAFF8C0EEF6E0BCFE9FF0CCFC2
:1014F000EAFFEF6A000E0B19146E0CCF15F0010E07
:1015000014C0DBFF020E15C0DBFF010EDBCFE9FFCD
:10151000020EDBCFEAFFEF6A030EE15C02E2E16A52
:10152000E552E16EE552E7CFD9FF120004011051F8
:10153000600BE842E842E842E842E842000901E084
:101540004CD011510C0A48E00B0A43E00C0A35E07C
:10155000010A26E00B0A22E0020A20E0030A1CE04E
:10156000080A10E0010A0CE00F0A08E0030A01E093
:1015700033D00F01148F080E006F2FD0B5D82DD0A7
:101580002BDB2BD00F01010E116F0F0E126F148188
:10159000010E156F148F21D048D91FD01FD81DD030
:1015A00014510F01116F126B020E11270F0E12232F
:1015B0001481010E156F148F10D00F01148F0401C8
:1015C0001451EA6A020FE96E0F0EEA2212C4EFFF0D
:1015D00004D08BEC1CF001D000D01200D9CFE6FF74
:1015E000E1CFD9FF050EE1260401120510E11051EB
:1015F0001F0B00090CE10F01148F030E0401115D94
:1016000004E10F01010E196F02D00F01196B0401E3
:10161000125160E110511F0B02085CE114510F0BD5
:10162000000958E00F01148F040EDB6A020EF36EFE
:10163000040EDBCFF4FFF350F45C4CE2000EDE6EE0
:10164000040EDD6E04011451800B01E0010E166ED4
:1016500014510F0BE8241624040DF3CF14F0F4CF2B
:1016600015F0D9CFE9FFDACFEAFF1450EE26155076
:10167000ED22030E115D07E1DECFE9FFDDCFEAFFCA
:10168000840EEF6E24D014510F0B156A4C0F146E9C
:101690000F0E1522020E14C0DBFF030E15C0DBFF78
:1016A000020EDBCFE9FF030EDBCFEAFFEE90ED5237
:1016B00014AF07D0DECFE9FFDDCFEAFF400EEF6EBB
:1016C00006D0DECFE9FFDDCFEAFFC80EEF6E040ED5
:1016D000DB2AACD7050EE15C02E2E16AE552E16E7D
:1016E000E552E7CFD9FF1200800E0401105D01E042
:1016F0009BD00F01C00E146F04011351030A56E072
:10170000010A10E0030A03E00F01146B8DD00F01F2
:10171000480E116F390E126F000E136F120E156FF7
:10172000166B82D0EC0E146E390E156E000E166E0E
:1017300012C417F0186A196A030E0C6E0D6A0E6A4D
:1017400017C007F018C008F019C009F04BEC1DF0E5
:1017500004C017F005C018F006C019F01450172483
:10176000F36E15501820F46E16501920F86EF4CF51
:10177000F7FFF3CFF6FF0900F5CF11FF0900F5CF12
:1017800012FF0800F5CF13FF11CFF6FF12CFF7FFBE
:1017900013CFF8FF020EF626000EF722F8220900FA
:1017A000F5CF15FF0A00F5CF16FF3ED0EF0E146EF1
:1017B000390E156E000E166E12C417F0186A196AEB
:1017C000030E0C6E0D6A0E6A17C007F018C008F001
:1017D00019C009F04BEC1DF004C017F005C018F05B
:1017E00006C019F014501724F36E15501820F46E2B
:1017F00016501920F86EF4CFF7FFF3CFF6FF09006B
:10180000F5CF11FF0900F5CF12FF0800F5CF13FF48
:1018100011CFF6FF12CFF7FF13CFF8FF0800F550F6
:101820000F01156F166B00D01200D9CFE6FFE1CF84
:10183000D9FF020EE1260401186B196B10511F0B22
:10184000020A12E0030A0DE0010A01E034D00F01A0
:10185000148F040118810F01190502E10401188396
:101860002AD00F01148F27D00F01148F000EDE6EC7
:10187000040EDD6E04011451800B01E0010E166EA2
:1018800014510F0BE8241624040DF3CF14F0F4CFF9
:1018900015F0D9CFE9FFDACFEAFF1450EE26155044
:1018A000ED22DECFE9FFDDCFEAFFEF50040B02E0CF
:1018B000010E186F00D00F0114AF07D0180E116F72
:1018C000040E126F1481020E156F020EE15C02E22B
:1018D000E16AE552E16EE552E7CFD9FF1200659863
:1018E0000F0114BF20D005CFE9FF06CFEAFFEE526B
:1018F000080EEF6E05CFE9FF06CFEAFF020EE926DC
:10190000000EEA22100EEE6E040EED6E05CFE9FF1A
:1019100006CFEAFF8C0EEF6E0BCFE9FF0CCFEAFF8C
:10192000840EEF6E81D0040110AF56D00F01155117
:101930000401165D0F0116510401175904E216C483
:1019400015FF17C416FF71D80F01010E106F05CFD8
:10195000E9FF06CFEAFFEE52080EEF6E05CFE9FF72
:1019600006CFEAFF020EE926000EEA22100EEE6E06
:10197000040EED6E05CFE9FF06CFEAFF800EEF6E95
:1019800003CFE9FF04CFEAFFEE52080EEF6E03CF5C
:10199000E9FF04CFEAFF020EE926000EEA22100E4C
:1019A000EE6E040EED6E03CFE9FF04CFEAFF800E6A
:1019B000EF6E0BCFE9FF0CCFEAFF020EE926000E17
:1019C000EA22180EEE6E040EED6E0BCFE9FF0CCF7F
:1019D000EAFFC80EEF6E28D00F01020E106F0BCF7A
:1019E000E9FF0CCFEAFFEE52EF6A0BCFE9FF0CCF15
:1019F000EAFFC80EEF6E05CFE9FF06CFEAFFEE5211
:101A0000080EEF6E05CFE9FF06CFEAFF020EE926CA
:101A1000000EEA22180EEE6E040EED6E05CFE9FF01
:101A200006CFEAFFC80EEF6E1200D9CFE6FFE1CF76
:101A3000D9FF020EE1260F01080E155D000E1659A2
:101A40000EE215CFDEFF16CFDDFF0F5103E1010ED1
:101A50000F6F04D00F0502E1020E0F6F03D0080EC6
:101A6000DE6EDD6A0BCFE9FF0CCFEAFFEF920BCF02
:101A7000E9FF0CCFEAFFEF900BCFE9FF0CCFEAFFB5
:101A8000010EDB50EF120BCFE9FF0CCFEAFFEE5255
:101A9000DFCFEFFF000EDB50155F010EDB50165B52
:101AA000180E176F040E186F14B124D0D9CFE9FFA8
:101AB000DACFEAFFEE50ED101CE011CFF6FF112B4C
:101AC00012CFF7FF000E122313CFF8FF13230800E5
:101AD000F550E66E17CFE9FF18CFEAFF172B000E7F
:101AE0001823E552E750EF6EDF06010E01E2DB0638
:101AF000DDD71FD0D9CFE9FFDACFEAFFEE50ED10E6
:101B000018E011CFE9FF12CFEAFF112B000E1223CC
:101B1000EF50E66E17CFE9FF18CFEAFF172B000E44
:101B20001823E552E750EF6EDF06010E01E2DB06F7
:101B3000E1D7020EE15C02E2E16AE552E16EE552B4
:101B4000E7CFD9FF1200D9CFE6FFE1CFD9FF020ED0
:101B5000E12605CFE9FF06CFEAFFEF50030BE76E62
:101B6000010EE7CFDBFF05CFE9FF06CFEAFFEE521C
:101B7000EFCFDFFFDE500F011527DD501623180EC3
:101B8000116F040E126FD9CFE9FFDACFEAFFEE50E2
:101B9000ED1018E011CFE9FF12CFEAFF112B000E74
:101BA0001223EF50E66E17CFE9FF18CFEAFF172B8D
:101BB000000E1823E552E750EF6EDF06010E01E23A
:101BC000DB06E1D7020EE15C02E2E16AE552E16E7A
:101BD000E552E7CFD9FF12000F01148F0F0EE66E0A
:101BE000E66AE66A4D0EE66E0F0EE66EB7EC1DF085
:101BF000146E050EE15E1450010EE66EE66AE66AAA
:101C0000020EE66E0F0EE66EB7EC1DF0146E050EBA
:101C1000E15E145012C401FF0401125104E10F01EE
:101C2000100E006F05D00F01200E006F8CEC1CF021
:101C30001200D9CFE6FFE1CFD9FF020EE126000E58
:101C4000DE6E040EDD6EFD0EDB50040DF3CF16F0DC
:101C5000FE0EDB50080DF3501624146E156A020EAA
:101C60000F0B05E0D89015321432E806FBE1D8904E
:101C700014361536D89014361536D9CFE9FFDACF99
:101C8000EAFF1450EE261550ED22DECFE9FFDDCF3E
:101C9000EAFFEF9EFD0EDB500FE1FE0EEA6ADB3439
:101CA000FE0BEA36E96E070EE9260F0EEA22DECFBA
:101CB000EEFFDDCFEDFF0ED0FE0EEA6ADB34FE0B49
:101CC000EA36E96E0B0EE9260F0EEA22DECFEEFFB2
:101CD000DDCFEDFFDECFE9FFDDCFEAFFEF8C020EB7
:101CE000E15C02E2E16AE552E16EE552E7CFD9FF3D
:101CF0001200D9CFE6FFE1CFD9FF020EE126FE0E9A
:101D0000DB50156A4C0F146E0F0E152214C0DEFF47
:101D100015C0DDFFFD0EDB50E66EDECFE9FFDDCF47
:101D2000EAFFE552E750EE6EED6AFD0EDBA407D048
:101D3000E66AFE0EDBCFE6FF7CDFE552E552FD0EE4
:101D4000DBA208D0010EE66EFE0EDBCFE6FF71DFF0
:101D5000E552E552020EE15C02E2E16AE552E16E13
:101D6000E552E7CFD9FF1200D9CFE6FFE1CFD9FF87
:101D7000020EE126FD0EDBCFE6FFFE0EDB50E8246F
:101D8000E552E724040DF3CF14F0F4CF15F0000E64
:101D90001426040E152214C0DEFF15C0DDFF840ECC
:101DA000146EDECFE9FFDDCFEAFF1450EF12020E12
:101DB000E15C02E2E16AE552E16EE552E7CFD9FF6C
:101DC0001200D9CFE6FFE1CFD9FF020EE126FD0ECA
:101DD000DB500FE0FE0EEA6ADB34FE0BEA36E96EFA
:101DE0000B0EE9260F0EEA22EECFDEFFEDCFDDFF70
:101DF0000ED0FE0EEA6ADB34FE0BEA36E96E070E01
:101E0000E9260F0EEA22EECFDEFFEDCFDDFFDECFBB
:101E1000E9FFDDCFEAFFEF7CDECFE9FFDDCFEAFFB0
:101E2000020EE926000EEA22FB0EDBCFEEFFFC0ECF
:101E3000DBCFEDFFDECFE9FFDDCFEAFFEE52FA0E9A
:101E4000DBCFEFFF400E146EDECFE9FFDDCFEAFF00
:101E50001450EF16880E146EDECFE9FFDDCFEAFFD7
:101E60001450EF12FD0EDB500BE0FE0EEA6ADB347D
:101E7000FE0BEA36E96E0B0EE9260F0EEA220AD0B7
:101E8000FE0EEA6ADB34FE0BEA36E96E070EE9263F
:101E90000F0EEA22DECF14F0DDCF15F014C0F3FFF1
:101EA00015C0F4FF020EE15C03E200D0E16AE552E6
:101EB000E16EE552E7CFD9FF1200D9CFE6FFE1CFBF
:101EC000D9FF010EF36EFC0EDB5004E0D890F33620
:101ED000E806FCE1F350E81C146EFD0EDBCFE9FFD1
:101EE000FE0EDBCFEAFF1450EF16E552E7CFD9FF25
:021EF0001200DE
:0E1EF2008150100B100A01E0010E00D012000A
:101F0000F36A020EF46E00D0120029CF06F02ACF39
:101F100007F02BCF08F02CCF09F000D012009388E7
:101F20008186939692881200D9CFE6FFE1CFD9FF40
:101F3000050EE126010EF36E020EF3CFDBFF818664
:101F4000800EE66EE66A020EE66E7CEC16F0E55256
:101F5000E552E552640EE66E2EEC15F0E552DE6AAF
:101F6000DD6ADECF14F0DDCF15F00A0E145C000E32
:101F7000155809E2E668ACEC16F0E552DF2A010ECE
:101F800001E3DB2AEED78196010EE66E2EEC15F00A
:101F9000E552E66AE66AE66AE66AE66AA7D8146E79
:101FA000050EE15E1450030EF3CFDBFF040EF4CFF9
:101FB000DBFF030EDB50FF0805E0030EDB50F70BE1
:101FC000010805E0020EDB6A8186DB507FD0DE6807
:101FD0000F0EDD6EE66AE66AE66AE66A010EE66EF6
:101FE00085D8146E050EE15E1450030EF3CFDBFFAF
:101FF000040EF4CFDBFFDF06010E01E2DB06030E69
:10200000DB5007E0D9CFE9FFDACFEAFFEE50ED1061
:10201000E1E1D9CFE9FFDACFEAFFEE50ED1004E1BC
:10202000020EDB6A81864FD0800EE66EE66AE66AB3
:102030007CEC16F0E552E552E552E66AE66AE66A9D
:10204000E66A160EE66E52D8146E050EE15E145066
:10205000030EF3CFDBFF040EF4CFDBFFE66A020EC4
:10206000E66EE66AE66A060EE66E40D8146E050E67
:10207000E15E1450DE68DD6AD9CFE9FFDACFEAFF0E
:10208000000ED880EE54000EED5413E2000EE66E02
:10209000E66AE66AE66AE66AE66ADBD9146E060E66
:1020A000E15E1450010805E0DF06010E01E2DB06E7
:1020B000E3D7D9CFE9FFDACFEAFFEE50ED1003E125
:1020C000020EDB6A8186020EDB5000D0146E050E14
:1020D000E15C02E2E16AE552E16E1450E552E7CFBD
:1020E000D9FF1200C0EC16F081861200D9CFE6FFAE
:1020F000E1CFD9FF0B0EE126080EDE6EDD6A819678
:10210000A20E146E3B0E156E000E166EFE0EDBCF89
:1021100017F0186A196A020ED89017361836193651
:10212000E806FAE114501724F36E15501820F46EE7
:1021300016501920F86EF4CFF7FFF3CFF6FF080022
:102140000A0EF5CFDBFFD950FA0FE96EFF0EDA2049
:10215000EA6E060EEECFDBFF070EEECFDBFF080EBA
:10216000EECFDBFF090EEECFDBFFA20E146E3B0EAF
:10217000156E000E166EFE0EDBCF17F0186A196A88
:10218000020ED890173618361936E806FAE11450C0
:102190001724F36E15501820F46E16501920F86E9F
:1021A000F4CFF7FFF3CFF6FFF62A000EF722F8225E
:1021B0000800050EF5CFDBFF0A0EDB8CDBCFE6FF58
:1021C000ACEC16F0E552090EDBCFE6FFACEC16F0F6
:1021D000E552080EDBCFE6FFACEC16F0E552070E39
:1021E000DBCFE6FFACEC16F0E552060EDBCFE6FFE8
:1021F000ACEC16F0E552050EDBCFE6FFACEC16F0CA
:10220000E552A20E146E3B0E156E000E166EFE0EFB
:10221000DBCF17F0186A196A020ED89017361836F5
:102220001936E806FAE114501724F36E15501820F9
:10223000F46E16501920F86EF4CFF7FFF3CFF6FFC7
:10224000020EF626000EF722F8220800F55028E0CC
:10225000A20E1A6E3B0E1B6E000E1C6EFE0EDBCF26
:102260001DF01E6A1F6A020ED8901D361E361F36DC
:10227000E806FAE11A501D24F36E1B501E20F46E7E
:102280001C501F20F86EF4CFF7FFF3CFF6FF020EBD
:10229000F626000EF722F8220800F550010816E194
:1022A0006EEC15F0E76E030EE7CFDBFFDF06010EE5
:1022B00001E2DB06030EDB50FF0807E1D9CFE9FF9F
:1022C000DACFEAFFEE50ED10EBE133D0A20E146E40
:1022D0003B0E156E000E166EFE0EDBCF17F0186A61
:1022E000196A020ED890173618361936E806FAE140
:1022F00014501724F36E15501820F46E1650192040
:10230000F86EF4CFF7FFF3CFF6FF020EF626000EBD
:10231000F722F8220800F55002080BE1DFDBDEDBD4
:10232000E76E040EE7CFDBFFD9DBE76E030EE7CFE6
:10233000DBFFA20E146E3B0E156E000E166EFE0E27
:10234000DBCF17F0186A196A020ED89017361836C4
:102350001936E806FAE114501724F36E15501820C8
:10236000F46E16501920F86EF4CFF7FFF3CFF6FF96
:10237000020EF626000EF722F8220800F55001089A
:1023800027E1030EDB6A020EDB6AFF0EF36E020E1C
:10239000DBCFF4FFF350F45C1BE2030EDB5018E1DB
:1023A000DE68DD689BDBE76E030EE7CFDBFFDF0651
:1023B000010E01E2DB06030EDB5007E1D9CFE9FF96
:1023C000DACFEAFFEE50ED10EDE1020EDB2ADDD7A9
:1023D000E668ACEC16F0E552A20E146E3B0E156EDC
:1023E000000E166EFE0EDBCF17F0186A196A020E89
:1023F000D890173618361936E806FAE11450172423
:10240000F36E15501820F46E16501920F86EF4CFA4
:10241000F7FFF3CFF6FF030EF626000EF722F822A1
:102420000800F55001E18186030EDBCF14F0040EA5
:10243000DBCF15F014C0F3FF15C0F4FF0B0EE15C09
:1024400003E200D0E16AE552E16EE552E7CFD9FF41
:102450001200D9CFE6FFE1CFD9FF140EE126010E1D
:10246000F36E070EF3CFDBFFFB0EDBCF14F0FC0E99
:10247000DBCF15F0FD0EDBCF16F0FE0EDBCF17F035
:10248000090E1F0B07E0D89014361536163617368E
:10249000E806F9E1080E14C0DBFF090E15C0DBFFEA
:1024A0000A0E16C0DBFF0B0E17C0DBFFD950080F5A
:1024B000E96EDACFEAFFEECFE6FFEECFE6FFEECF32
:1024C000E6FFEFCFE6FF070EE66E10DE146E050E98
:1024D000E15E1450040EF3CFDBFF050EF4CFDBFFFB
:1024E000040EDB501FE0D950080FE96EDACFEAFF87
:1024F000EECFE6FFEECFE6FFEECFE6FFEFCFE6FF53
:10250000070EE66EF3DD146E050EE15E1450040E48
:10251000F3CFDBFF050EF4CFDBFF040EDB5002E050
:10252000000ECFD1DE68020EDD6E400EF36E020E9D
:10253000F3CFDBFF030EDB6AD950020FE96EDACF6F
:10254000EAFFEE50ED1006E0020EDB06030E01E29C
:10255000DB06F2D7C3DAE76E060EE7CFDBFFDF0656
:10256000010E01E2DB06400EF36E020EF3CFDBFF3D
:10257000030EDB6AD950020FE96EDACFEAFFEE50A4
:10258000ED1006E0020EDB06030E01E2DB06F2D7D9
:10259000060EDB50FF0807E1D9CFE9FFDACFEAFFEB
:1025A000EE50ED10D7E1D9CFE9FFDACFEAFFEE50D8
:1025B000ED1004E0060EDB50FE0803E0070EDB6AB8
:1025C00079D1FB0EDBCF14F0FC0EDBCF15F0FD0E46
:1025D000DBCF16F0FE0EDBCF17F0145015101610DF
:1025E00017100EE1D950F90FE96EFF0EDA20EA6EEE
:1025F000EE50ED1005E10F01296B2A6B2B6B2C6B54
:10260000DE6ADD6ADECF14F0DDCF15F0000E145C5B
:10261000020E155801E348D1D950F90FE96EFF0EAB
:10262000DA20EA6EEE50ED1012E058DAE66EF90E9E
:10263000DBCF14F0FA0EDBCF15F0DE501424E96E78
:10264000DD501520EA6EE552E750EF6E28D1FB0E03
:10265000DBCF14F0FC0EDBCF15F0FD0EDBCF16F058
:10266000FE0EDBCF17F0145015101610171001E0F6
:1026700015D1D9CFE9FFDACFEAFFC60EEE1802E195
:10268000010EED1801E008D129DA146E0C0E14C009
:10269000DBFF0D0EDB6A0E0EDB6A0F0EDB6A1EDA45
:1026A000146E156A166A176A080E1F0B07E0D89099
:1026B0001436153616361736E806F9E1D9500C0FE0
:1026C000E96EDACFEAFF1450EE121550EE121650F2
:1026D000EE121750EE1202DA146E156A166A176AB5
:1026E000100E1F0B07E0D890143615361636173625
:1026F000E806F9E1D9500C0FE96EDACFEAFF145081
:10270000EE121550EE121650EE121750EE12E6D9D8
:10271000146E156A166A176A180E1F0B07E0D89018
:102720001436153616361736E806F9E1D9500C0F6F
:10273000E96EDACFEAFF1450EE121550EE12165081
:10274000EE121750EE12CAD9146E100E14C0DBFF31
:10275000110EDB6A120EDB6A130EDB6ABFD9146E30
:10276000156A166A176A080E1F0B07E0D890143610
:10277000153616361736E806F9E1D950100FE96E0E
:10278000DACFEAFF1450EE121550EE121650EE1288
:102790001750EE12A3D9146E156A166A176A100E36
:1027A0001F0B07E0D8901436153616361736E80694
:1027B000F9E1D950100FE96EDACFEAFF1450EE12AA
:1027C0001550EE121650EE121750EE1287D9146EF5
:1027D000156A166A176A180E1F0B07E0D890143690
:1027E000153616361736E806F9E1D950100FE96E9E
:1027F000DACFEAFF1450EE121550EE121650EE1218
:102800001750EE12080EDE26000EDD22100EDBCF72
:1028100014F0110EDBCF15F0120EDBCF16F0130EF5
:10282000DBCF17F0D9500C0FE96EDACFEAFFEE508C
:102830001426EE501522EE501622EE501722145098
:102840000F01295D15502A5916502B5917502C5934
:1028500022E20C0EDBCF14F00D0EDBCF15F00E0EC6
:10286000DBCF16F00F0EDBCF17F0D950100FE96E4B
:10287000DACFEAFF1450EE24296F1550EE202A6FAC
:102880001650EE202B6F1750EE202C6F2907000EEC
:102890002A5B2B5B2C5B01D021D901D01FD9DF2A09
:1028A000010E01E3DB2AAED6E66856DAE552E668A9
:1028B00053DAE552E66850DAE5528186070EDB50BE
:1028C00000D0146E140EE15C02E2E16AE552E16EA2
:1028D0001450E552E7CFD9FF1200D9CFE6FFE1CF80
:1028E000D9FF060EE126010EF36E050EF3CFDBFFD6
:1028F000FB0EDBCF14F0FC0EDBCF15F0FD0EDBCFB3
:1029000016F0FE0EDBCF17F014501510161017102E
:1029100006E1F80EDB5003E1050EDB6A8AD0FB0E00
:10292000DBCF14F0FC0EDBCF15F0FD0EDBCF16F085
:10293000FE0EDBCF17F0090E1F0B07E0D890143600
:10294000153616361736E806F9E114C0E6FF15C04D
:10295000E6FF16C0E6FF17C0E6FF090EE66E76EC4E
:1029600010F0186E050EE15E1850030EF3CFDBFF7A
:10297000040EF4CFDBFF030EDB5003E0050EDB6A31
:1029800057D0FE0EE66EE8D9E552DE6ADD6ADECF8C
:1029900014F0DDCF15F0000E145C020E155815E290
:1029A000F90EDBCF14F0FA0EDBCF15F0DE50142455
:1029B000E96EDD501520EA6EEF50E66ECDD9E55296
:1029C000DF2A010E01E3DB2AE2D7E668C5D9E5522A
:1029D000E668C2D9E55282D8E76E020EE7CFDBFF88
:1029E000DB500F0B050803E0050EDB6A1ED0DE6A24
:1029F000DD6A74D8E76E020EE7CFDBFFDF2A010E37
:102A000001E3DB2A020EDB5007E1D9CFE9FFDACF81
:102A1000EAFFEE50ED10EDE1D9CFE9FFDACFEAFFA2
:102A2000EE50ED1002E1050EDB6AE66895D9E5523D
:102A30008186050EDB50146E060EE15C03E200D0C9
:102A4000E16AE552E16E1450E552E7CFD9FF12007A
:102A50008050100B01E0010E00D01200D9CFE6FF2C
:102A6000E1CFD9FF050EE126FE0EDB50DF6EDF5011
:102A7000DF06000927E06C0EF36E010EF3CFDBFFDB
:102A8000020EF36E020EF3CFDBFF030EDB6A040EC1
:102A9000DB6AD950010FE96EDACFEAFFEFCF14F00D
:102AA000EE06000EEFCF15F0EE5AEFCF16F0EE5A0D
:102AB000EFCF17F0EF5A145015101610171001E051
:102AC000E8D7D5D7000000D0050EE15C02E2E16A4C
:102AD000E552E16EE552E7CFD9FF1200C968C7A001
:102AE000FED7C95000D01200D9CFE6FFE1CFD9FF01
:102AF000FB0EDBCF14F0FC0EDBCF15F0FD0EDB5030
:102B00001424E96EFE0EDB501520EA6EEF5000D063
:102B1000E552E7CFD9FF1200D9CFE6FFE1CFD9FFC9
:102B2000040EE126FB0EDBCF14F0FC0EDBCF15F01C
:102B3000FD0EDB501424E96EFE0EDB501520EA6E0C
:102B4000EFCFDFFF010EE76EFB0EDBCF14F0FC0EC4
:102B5000DBCF15F0E7501426000E1522FD0EDB50DA
:102B60001424E96EFE0EDB501520EA6E010EEFCF45
:102B7000DBFFDB50E66ED950020FE96EDACFEAFFD9
:102B8000E552E750EE6EED6AD950020FE96EDACFEA
:102B9000EAFFEE50ED6EEF6ADF50146E156AD95001
:102BA000020FE96EDACFEAFF1450EE121550ED1263
:102BB000020EDBCF14F0030EDBCF15F014C0F3FFD1
:102BC00015C0F4FF040EE15C03E200D0E16AE552B7
:102BD000E16EE552E7CFD9FF1200D9CFE6FFE1CF92
:102BE000D9FF080EE126FB0EDBCFE6FFFC0EDBCFA4
:102BF000E6FFFD0EDBCFE6FFFE0EDBCFE6FF8CDF50
:102C0000E552E552E552E552F3CFDEFFF4CFDDFFAA
:102C1000020EE76EFB0EDBCF14F0FC0EDBCF15F0DF
:102C2000E7501426000E152214C0E6FF15C0E6FF7B
:102C3000FD0EDBCFE6FFFE0EDBCFE6FF6DDFE552DC
:102C4000E552E552E552020EF3CFDBFF030EF4CF5F
:102C5000DBFF020EDBCF14F0030EDBCF15F0040E0A
:102C600014C0DBFF050E15C0DBFF060EDB6A070E86
:102C7000DB6AD950040FE96EDACFEAFF100EE76E77
:102C8000D890EF36010EEB36020EEB36030EEB3624
:102C9000E706F6E1DECF14F0DDCF15F0166A176A0D
:102CA000D950040FE96EDACFEAFF1450EE12155036
:102CB000EE121650EE121750EE12040EDBCF14F087
:102CC000050EDBCF15F0060EDBCF16F0070EDBCFBF
:102CD00017F014C006F015C007F016C008F017C0B2
:102CE00009F0080EE15C03E200D0E16AE552E16E12
:102CF000E552E7CFD9FF1200D9CFE6FFE1CFD9FFE8
:102D00003F0EC716C66AFE0EDB50C612FC0EDB5025
:102D1000C712FD0EDB50030A0AE0010A05E0020AB1
:102D200001E007D0C78C05D0C78CC68802D0C68802
:102D300000D0FE0EDB50050A05E0010A02E0949681
:102D400004D093869486C79E00D0949A9488C68AAD
:102D5000E552E7CFD9FF1200D9CFE6FFE1CFD9FF87
:102D6000FE0EDB50C96EC6AE03D0FF0E05D002D0FA
:102D7000C7A0FED7000E00D0E552E7CFD9FF120062
:042D8000C69A1200DD
:0C2D84000001976B986B400EE66E200E6D
:102D9000E66E040EE66EE66A010EE66EE1EC0EF0FB
:102DA000146E050EE15E1450F3CF95F0F4CF96F05B
:102DB0000001606BA36BA46BA56BA66BA76BA86BE4
:102DC000A96BAA6B9B6B9C6B6E6B010E6E5D1FE219
:102DD00079EC0FF0000916E094EC0FF0000912E016
:102DE000010E6EC0E7FFE75204E0E846FE0BE7067F
:102DF000FCE1146E156A14BE1568145000019B1393
:102E000015509C131FEC1CF000016E2BDED7120036
:102E100004011151FE0A04E0010A01E00ED00DD0B8
:102E20000401186B0F01180E116F040E126F010EC2
:102E3000156F166BC10E146F00D01200D9CFE6FFCC
:102E4000E1CFD9FFE65200016051030A01E1A9D0A8
:102E5000010A01E195D0030A01E18BD0010A01E0EA
:102E6000E9D09551961102E1000E08D095C0E9FF16
:102E700096C0EAFFEF50800B01E0010E000901E06F
:102E800077D020C461F021C462F022C463F023C46F
:102E900064F024C465F025C466F026C467F027C436
:102EA00068F028C469F029C46AF02AC46BF02BC406
:102EB0006CF02CC46DF02DC46EF02EC46FF0DF6A80
:102EC00004012E51DF5C13E2DF50EA6A2F0FE96E36
:102ED000040EEA22EF50E66EDF50EA6A700FE96EE8
:102EE000000EEA22E552E750EF6EDF2AE9D795C0DF
:102EF000E9FF96C0EAFFEE52EFCF80F01F0E00010F
:102F0000805D36E1550E611908E1530E621905E145
:102F1000420E631902E1430E64192AE16E510F0853
:102F200027E36F51100824E3010E6F5D21E36D511B
:102F300003E0800E6D5D1CE165C043F466C044F49F
:102F400067C045F468C046F40401550E3F6F530E48
:102F5000406F420E416F530E426F800E00016D5D57
:102F600003E1010E606F04D06D5102E1020E606F4B
:102F700061D060DAFF0803E10001030E606F5AD0F0
:102F800059DAFF080DE104014B5107E1475148119F
:102F900049114A1102E0020E4B6F0001030E606FEF
:102FA00049D09751981102E1000E08D097C0E9FF6F
:102FB00098C0EAFFEF50800B01E0010E000901E02C
:102FC00039D00D0EE66E3F0EE66E040EE66E010E73
:102FD000E66EE66EE1EC0EF0146E050EE15E145046
:102FE000F3CF97F0F4CF98F000019551961102E1DC
:102FF000000E08D095C0E9FF96C0EAFFEF50800BA5
:1030000001E0010E000913E11F0EE66E200EE66ED0
:10301000040EE66EE66A010EE66EE1EC0EF0146E4A
:10302000050EE15E1450F3CF95F0F4CF96F0000159
:10303000606B00D00001605100D0E552E552E7CF4F
:10304000D9FF1200D9CFE6FFE1CFD9FF090EE12663
:103050000F012D51FE0A01E128D1030A01E1FAD046
:10306000D20A01E1EED0340A01E1EBD01B0A01E102
:10307000D4D01E0A01E1B8D0040A01E1A4D0190A93
:1030800001E17AD0290A72E0020A6AE00D0A26E01C
:10309000370A06E0ED0A01E008D170C02DFF19D112
:1030A000240EE66EE66AFE0EE66E3B0EE66E000E3F
:1030B000E66E000EE66E060EE66E94EC1DF0146EE3
:1030C000070EE15E14500401240E476F486B496BF4
:1030D0004A6B4B6B0F01FD0E2D6FFBD004014B6B48
:1030E00085EC0FF0050E06C0DBFF060E07C0DBFF08
:1030F000070E08C0DBFF080E09C0DBFF80EC0FF0F5
:10310000F3CF14F0F4CF15F0010E14C0DBFF020E64
:1031100015C0DBFF030EDB6A040EDB6A080EDBCF93
:1031200000F6070EDBCF01F6060EDBCF02F6050E2A
:10313000DBCF03F6040EDBCF04F6030EDBCF05F680
:10314000020EDBCF06F6010EDBCF07F60401080EF8
:10315000476F486B496B4A6B0F01FD0E2D6FB9D05D
:10316000C2D9000902E10F012D69B3D088DA000944
:1031700002E10F012D69ADD0DF6ADF50146E156AD0
:10318000120E145C000E155813E2DF50EA6A810F2C
:10319000E96E000EEA22EF50E66EDF50EA6A000F99
:1031A000E96E060EEA22E552E750EF6EDF2AE5D718
:1031B0000401120E476F486B496B4A6B4B6B0F0152
:1031C000FD0E2D6F86D00601020E006F016B026BA3
:1031D000036B04014B6B040E476F486B496B4A6BE2
:1031E0000F01FD0E2D6F75D079EC0FF0000907E08F
:1031F00004014B6B476B486B496B4A6B0BD000016A
:1032000083918383839583973A0E8D6F8E6B040130
:10321000010E4B6F0F012D695CD0000183510F0B24
:10322000060806E104014B0503E10F012D6908D0F2
:1032300006DB0401476B486B496B4A6B0F012D6934
:1032400048D004014B6B476B486B496B4A6B0F01CD
:103250002D693FD000019751981102E1000E08D06E
:1032600097C0E9FF98C0EAFFEF50800B01E0010E24
:1032700000091AE147C4E6FF000EE66E060EE66E90
:10328000010EE66EE66EE1EC0EF0146E050EE15EE8
:103290001450F3CF97F0F4CF98F00F012D6904018B
:1032A000476B486B496B4A6B14D0C9DA00018381C4
:1032B000839383858397200E8D6F8E6B0401010E9F
:1032C0004B6F476B486B496B4A6B0F01FD0E2D6FBF
:1032D00000D0090EE15C02E2E16AE552E16EE552DE
:1032E000E7CFD9FF1200D9CFE6FFE1CFD9FFE652F1
:1032F0000F012D51FD0A6EE0020A69E0ED0A49E076
:103300000C0A41E01E0A3FE0030A0DE0010EE66EE2
:10331000E66EB4EC0EF0E552E5520401010E4B6F7F
:103320000F012D6982D08BDA00018391838383950D
:1033300083973A0E8D6F8E6BDF6ADF50146E156ABD
:10334000120E145C000E155813E2DF50EA6A810F6A
:10335000E96E000EEA22EF50E66EDF50EA6A000FD7
:10336000E96E060EEA22E552E750EF6EDF2AE5D756
:103370000401120E476F486B496B4A6B4B6B0F0190
:10338000FD0E2D6F52D00401010E4B6F0F012D6900
:103390004CD0240EE66EE66AFE0EE66E3B0EE66E3E
:1033A000000EE66E000EE66E060EE66E94EC1DF064
:1033B000146E070EE15E14500401240E476F486B33
:1033C000496B4A6B4B6B0F01FD0E2D6F2ED070C0F9
:1033D0002DFF2BD000019751981102E1000E08D06B
:1033E00097C0E9FF98C0EAFFEF50800B01E0010EA3
:1033F00000091AE147C4E6FF000EE66E060EE66E0F
:10340000010EE66EE66EE1EC0EF0146E050EE15E66
:103410001450F3CF97F0F4CF98F00F012D69040109
:10342000476B486B496B4A6B00D0E552E552E7CFDA
:10343000D9FF120079EC0FF0000915E1010E6EC002
:10344000E7FFE75204E0E846FE0BE706FCE1E81C74
:10345000146E156A14BE1568145000019B171550A0
:103460009C1741DF3CD0010E6EC0E7FFE75204E03D
:10347000E846FE0BE706FCE1166E176A16BE1768F3
:1034800000019B511614146E9C511714156E1450A4
:10349000151024E194EC0FF000091EE0010E6EC03F
:1034A000E7FFE75204E0E846FE0BE706FCE1146E96
:1034B000156A14BE1568145000019B1315509C1317
:1034C0008391838383858397280E8D6F8E6B040190
:1034D000010E4B6FB7DD01D006DF01D0B3DD0F0168
:1034E0002D5100D012000F012E51040A01E17CD0B1
:1034F000070A6DE0010A27E0030A18E0010A01E06B
:10350000BAD072C0A2F073C0A1F074C0A0F075C0B0
:103510009FF077C09EF078C09DF004014B6B476B25
:10352000486B496B4A6B0F01010E2E6F00019D51D4
:103530009E1103E10F012E6B9ED09D07000E9E5B36
:103540000F01020E2E6F00019751981102E1000E3B
:1035500008D097C0E9FF98C0EAFFEF50800B01E068
:10356000010E000901E087D0000EE66E060EE66E41
:103570009FC0E6FFA0C0E6FFA1C0E6FFA2C0E6FF35
:1035800029EC12F0146E060EE15E145001080AE0F8
:103590000401010E4B6F476B486B496B4A6B00018E
:1035A000606F69D000019F2B000EA023A123A223EE
:1035B00004014B6B476B020E486F496B4A6B00016D
:1035C000000E936F060E946F0F01030E2E6F040111
:1035D0004751481149114A1104E10F01010E2E6FA4
:1035E0004AD00F01040E2E6F04014B5143E1400EEF
:1035F000475D000E4859000E4959000E4A593AE3FA
:1036000000019751981102E1000E08D097C0E9FF20
:1036100098C0EAFFEF50800B01E0010E000901E0C5
:103620002AD0400EE66E93C0E6FF94C0E6FF010E7E
:10363000E66EE66EE1EC0EF0146E050EE15E1450DF
:10364000F3CF97F0F4CF98F00F01030E2E6F400EDA
:103650000001695F000E6A5B6B5B6C5B400E0401EE
:10366000475F000E485B495B4A5B400E00019327B1
:10367000000E942300D00F012E5100D012000F0134
:103680002F51020A01E1B5D0060A74E0070A2BE0C7
:10369000020A14E0010A01E0CED072C0A2F073C0A9
:1036A000A1F074C0A0F075C09FF077C09EF078C004
:1036B0009DF004014B6B0001010E606F00019D51F4
:1036C0009E1103E10F012F6BB6D00F01030E2F6F78
:1036D0000001000E936F060E946F0401476B020EFB
:1036E000486F496B4A6BD880000E04014755000EA5
:1036F0004855000E4955000E4A5528E200019551E3
:10370000961102E1000E08D095C0E9FF96C0EAFFCD
:10371000EF50800B01E0010E000901E08CD0400E5B
:10372000E66E93C0E6FF94C0E6FFE66A010EE66E21
:10373000E1EC0EF0146E050EE15E1450F3CF95F03F
:10374000F4CF96F00F01040E2F6F14D028EC15F073
:1037500000090CE000018391838383958397270EF2
:103760008D6F8E6B0401010E4B6F03D00F01020EA3
:103770002F6F61D000019551961102E1000E08D023
:1037800095C0E9FF96C0EAFFEF50800B01E0010E03
:10379000000901E050D095C0E9FF96C0EAFFEE5263
:1037A000EFCF14F0156A166A176A1450695F155046
:1037B0006A5B16506B5B17506C5B95C0E9FF96C057
:1037C000EAFFEE52EFCF14F0156A166A176A14502A
:1037D0000401475F1550485B1650495B17504A5B20
:1037E000400E00019327000E94230F01030E2F6F4C
:1037F00022D0E66A000EE66E060EE66E9FC0E6FF79
:10380000A0C0E6FFA1C0E6FFA2C0E6FF6DEC14F089
:10381000146E070EE15E1450010801E00CD00001A7
:103820009F2B000EA023A123A2239D079E5B0F01C7
:10383000010E2F6F00D00F012F5100D01200000198
:1038400081918193819581978189818B818D819FE0
:10385000826B8391839383958397839B839D839FBF
:10386000846B856B866B876B0A0E886F896B8A6B9E
:103870008B6B8C6B8D6B8E6B8F6B906B916B926B7C
:02388000120034
:0E388200DACFE4FFE2CFDAFFE652E552E5CFFF
:10389000DAFF1100120005D878EC08F02BD8FCD71D
:1038A0001200D9CFE6FFE1CFD9FF020EE126580E74
:1038B000DE6E020EDD6E9B8CDFCF14F0DF06010E94
:1038C000DBCF15F001E2DB061450151001E0F4D750
:1038D000C088C168C268C0981CEC08F08FEC0FF07B
:1038E000020EE15C02E2E16AE552E16EE552E7CFE9
:1038F000D9FF1200200E0F01005D03E36550020B9B
:1039000001E002D01EEC17F01200120012001200AB
:10391000120008EF17F012001E0EE66E010EE66EA2
:1039200079EC0EF0E552E552C2EF16F065840F0116
:10393000080E306F070E316F3007000E315B3051CB
:083940003111FAE16594120057
:0839480012011001000000084B
:10395000D804090001000102000109022000010150
:1039600000C0320904000002080650000705810269
:10397000400000070501024000000403090434036D
:103980004D006900630072006F0063006800690009
:103990007000200054006500630068006E006F0036
:1039A0006C006F0067007900200049006E00630022
:1039B0002E003A034D006900630072006F0063003F
:1039C00068006900700020004D0061007300730002
:1039D0002000530074006F007200610067006500F2
:1039E0002000440072006900760065005A39007AB0
:0839F00039007E3900B23900F4
:0839F8002A0EF66E100EF76EA8
:103A0000000EF86E0F010900F550246F0900F55003
:103A1000256F03E1246701D03DD00900F5501F6FE9
:103A20000900F550206F0900F550216F09000900C9
:103A3000F550E96E0900F550EA6E09000900090029
:103A4000F550226F0900F550236F09000900F6CFE9
:103A500026FFF7CF27FFF8CF28FF1FCFF6FF20CF95
:103A6000F7FF21CFF8FF0F01225302E1235307E0B4
:103A70000900F550EE6E2207F8E22307F9D726CFAA
:103A8000F6FF27CFF7FF28CFF8FF0F012407000E1E
:063A9000255BBFD7120008
:0A3A960009C013F008C012F007C0C9
:103AA00011F007500C02F4CF05F0F3CF04F00850EA
:103AB0000D02F4CF07F0F3CF06F00C02F350052609
:103AC000F4500622E86A072211500D02F350052631
:103AD000F4500622E86A072209500C02F350062629
:103AE000F450072209500D02086AE86A0822F350D0
:103AF0000726F450082211500E02F3500626F45007
:103B00000722096AE86A0822092212500E02F350BD
:103B10000726F4500822E86A092213500E02F350D7
:083B20000826F4500922000CF4
:083B2800FB0EE3CFF6FFFC0EDB
:103B3000E3CFF7FFFD0EE3CFF8FFFE0EE3CFE9FF83
:103B4000FF0EE3CFEAFFE9CFF3FFEACFF4FFF90E70
:103B5000E35003E1FA0EE35009E0F90EE30602E256
:103B6000FA0EE3060900F5CFEEFFF1D71200FE0EC4
:103B7000E3CFE9FFFF0EE3CFEAFFE9CFF3FFEACFA0
:103B8000F4FFFB0EE35003E1FC0EE35009E0FB0EF3
:103B9000E30602E2FC0EE306FD0EE350EE6EF1D703
:023BA000120011
:0E3BA2000095000001F9000009AF00010A1BA8
:103BB00000010CC300000DAF020010FF000011FF58
:103BC000000112FF000118FF000119FF000120FF92
:103BD000000021FF000022FF000023FF000024FF5F
:103BE000000025FF000026DF01003189010029E5E2
:0E3BF0000000377300003A2503003B2500005B
:023BFE00008045
:103C00000402200000004D6963726F6368704D61AB
:103C100073732053746F72616765202020203030E9
:023C2000303141
:0E3C22001EEE00F02EEE00F0F86A019CFCECA5
:0E3C30001CF01FEC1EF04BEC1CF0FBD712003A
:023C3E00120072
:033C4000FF000082
:020000040001F9
:01FFF800AA5E
:01FFF900F710
:01FFFA000501
:01FFFB00FF06
:01FFFD00F70C
:00000001FF
